:020000040000FA
:04000000CF303A289B
:08000800A000030EA100831209
:100010008B1C32288B1031181428B11C3228643004
:10002000010203183128182800001628172818285C
:1000300019281A281B281C281D281E281F283110A3
:10004000B114A810031005190314AA0DA90DA80DC9
:10005000B00B322831152A08AF002908AE00280855
:10006000AD00B11081010B11210E8300A00E200EF6
:02007000090085
:0C007400203084008001840A80300402E7
:10008000031C3C281230B0000A2283160C30850570
:1000900087018312850187010730990000309A009B
:1000A000103083168E008312603083168F00831207
:1000B0000030831691009F008312C83083168100A0
:1000C000831231309000003083168C008312103080
:1000D0008B00831600309B001C141A088312BC008E
:1000E000851D2A23831610309B001C141A088312C6
:1000F000BD00831630309B001C141A088312DE00EA
:100100000D2381018E018F010B118B100B108C01BF
:100110008B1798203119AE20B30B96280310851940
:100120000314B90DF03039020319662170238928B0
:100130006400311808000B1D08000B11B1103114B8
:100140001230B000051DA928321483160113831242
:100150000800321083160117831208003111013094
:10016000B7008B132030370783169B001C141A0826
:100170008312A400A500C030A506103037078316EF
:100180009B001C141A088312A30000303707831643
:100190009B001C141A088312A2008B17321CD6284D
:1001A00022090339A200A309A409A50922082D02E6
:1001B000031D602923082E02031D602924082F0235
:1001C000031D602901303702031DEB283D18EB2881
:1001D0003D143E14172202303702031DF428BD18C7
:1001E000F428BD143E14262203303702031DFD28D7
:1001F0003D19FD283D153E14322204303702031DFF
:100200000629BD190629BD153E143E2205303702C8
:10021000031D0F293D1A0F293D163E144D220630AD
:100220003702031D1829BD1A1829BD163E145C2279
:1002300007303702031D21293D1B21293D173E149C
:100240006B2208303702031D2A29BD1B2A29BD173E
:100250003E147A2209303702031D33295E183329F0
:100260005E143E1485220A303702031D3C29DE1835
:100270003C29DE143E1490220B303702031D452921
:100280005E1945295E153E149B220C303702031D72
:100290004E29DE194E29DE153E14A6220D303702F6
:1002A000031D57295E1A57295E163E14B1220E30DF
:1002B0003702031D6029DE1A6029DE163E14BC22B7
:1002C000B70A0F30370203180800B1280130B60012
:1002D000B300B400B500B70085018701B1139820C1
:1002E000B30BB629031085190314B90DF030390288
:1002F0000319DD29B40BB629013037020319C722CF
:10030000023037020319CC22033037020319D122FD
:10031000043037020319D622053037020319DB22D5
:10032000063037020319E022073037020319E522AD
:10033000083037020319EA22093037020319EF2285
:100340000A3037020319F4220B3037020319F9225D
:100350000C3037020319FE220D3037020319032334
:100360000E303702031908239630B400311D6F296F
:100370003111321CC0292D090339AD00AE09AF0976
:100380002F1CB1132F1C6F29B11B6F292E186F2939
:10039000B1178B1320303707BB002F08BA00F521A7
:1003A00010303707BB002E08BA00F52100303707A0
:1003B000BB002D08BA00F5218B1785018701B70A0C
:1003C000B6010F303702031C6F290D2308003E1CB5
:1003D00008003E101030BB003D08BA00F521303057
:1003E000BB005E08BA00F52108008B133A0883169B
:1003F0001C159A0083123B0883169B0055309D0004
:10040000AA309D009C1464009C18032A1C118312BE
:100410008B170800FF30C800CA15CB15CC15CD15B9
:10042000CE15CF15D015D115D215D31508008130B2
:10043000BD05FF30DE050130C405C0000030C2003C
:10044000C600BC185F14BC18DF1408008230BD055C
:10045000FF30DE050230C405C0000030C200C60017
:100460005F1008008430BD05FF30DE050630C4058E
:10047000C0000030C200C6005F1008008830BD0513
:10048000FF30DE050930C405C0000830C200C600D8
:10049000BC185F14BC18DF1408009030BD05FF3095
:1004A000DE051930C405C0000030C200C600BC180B
:1004B0005F14BC18DF140800A030BD05FF30DE0556
:1004C0002130C405C0000030C200C600BC185F1453
:1004D000BC18DF140800C030BD05FF30DE05103049
:1004E000C405C0000030C200C600BC185F14BC18B0
:1004F000DF140800FF30BD05C030DE055030C505F3
:10050000C1000030C300C70008007F30BD05C13006
:10051000DE052030C505C1000030C300C70008005B
:100520007F30BD05C230DE05E030C505C10020309A
:10053000C300C70008007F30BD05C430DE05503061
:10054000C505C1000030C300C70008007F30BD05ED
:10055000C830DE055030C505C1000030C300C700FB
:1005600008007F30BD05D030DE055030C505C10024
:100570000030C300C70008007F30BD05E030DE0555
:100580004030C505C1000030C300C700080010306E
:100590008506003087060800203085060030870673
:1005A00008002130850600308706080012308506D5
:1005B00000308706080012308506023087060800E2
:1005C00010308506043087060800003085060230AA
:1005D00087060800003085061130870608000030C5
:1005E00085062030870608000030850638308706EB
:1005F00008000030850611308706080000308506A7
:100600001130870608000030850611308706080083
:10061000003085063930870608003D181722BD18BE
:1006200026223D193222BD193E223D1A4D22BD1A05
:100630005C223D1B6B22BD1B7A225E188522DE18D0
:1006400090225E199B22DE19A6225E1AB122DE1AC2
:10065000BC220800B601B301B4013C1C322BBC0122
:10066000BC14342BBC013C143C08B6006400382B8D
:10067000392B3A2B3B2B3C2BFF30B41B8500B41F8E
:100680008501B30B362BB40B362B0310B60CB60812
:10069000031D362B0030BB003C08BA00F5210800D2
:1006A00005125C180516DC1C8512DC1885165C1D0D
:1006B00005105C190514DC1D8510DC1985145C1E01
:1006C00087105C1A8714DC1E0711DC1A07155C1FE3
:1006D00007105C1B0714DC1F8712DC1B8716080041
:1006E0008F08031908008F0178308E00C80FA22DE3
:1006F000C80A441CA02B461C912BCA1C822BCA0181
:100700004A15AE2B4A1D872BCA01CA15AE2BCA1D2E
:100710008C2BCA014A16AE2B4A1EAE2BCA01CA1434
:10072000AE2B4A1D962BCA014A16AE2BCA1D9B2B17
:10073000CA014A16AE2B4A1EAE2BCA01CA14AE2BF2
:10074000CA1CA52BCA014A15AE2B4A1DAA2BCA01E9
:10075000CA15AE2B4A1EAE2BCA014A15C41CD52B96
:10076000C61CC62BCB1CB72BCB014B15E32B4B1D4B
:10077000BC2BCB01CB15E32BCB1DC12BCB014B16D7
:10078000E32B4B1EE32BCB01CB14E32B4B1DCB2BCD
:10079000CB014B16E32BCB1DD02BCB014B16E32B00
:1007A0004B1EE32BCB01CB14E32BCB1CDA2BCB0161
:1007B0004B15E32B4B1DDF2BCB01CB15E32B4B1E36
:1007C000E32BCB014B15441D0A2C461DFB2BCC1CE7
:1007D000EC2BCC014C15182C4C1DF12BCC01CC155D
:1007E000182CCC1DF62BCC014C16182C4C1E182C9A
:1007F000CC01CC14182C4C1D002CCC014C16182C00
:10080000CC1D052CCC014C16182C4C1E182CCC01E0
:10081000CC14182CCC1C0F2CCC014C15182C4C1DB6
:10082000142CCC01CC15182C4C1E182CCC014C15BA
:10083000C41D402CC61D312CCD1C222CCD014D15C4
:100840005F134E2C4D1D272CCD01CD154E2CCD1DEB
:100850002C2CCD014D164E2C4D1E4E2CCD01CD1401
:100860004E2C4D1D362CCD014D164E2CCD1D3B2C46
:10087000CD014D164E2C4D1E4E2CCD01CD144E2CBF
:10088000CD1C452CCD014D154E2C4D1D4A2CCD01B6
:10089000CD154E2C4D1E4E2CCD014D155F1B772CCA
:1008A000441E772C461E682CCE1C592CCE014E15AA
:1008B000852C4E1D5E2CCE01CE15852CCE1D632CB5
:1008C000CE014E16852C4E1E852CCE01CE14852CC5
:1008D0004E1D6D2CCE014E16852CCE1D722CCE01D8
:1008E0004E16852C4E1E852CCE01CE14852CCE1C8A
:1008F0007C2CCE014E15852C4E1D812CCE01CE15A3
:10090000852C4E1E852CCE014E15C41EAC2CC61E49
:100910009D2CCF1C8E2CCF014F15BA2C4F1D932C24
:10092000CF01CF15BA2CCF1D982CCF014F16BA2C62
:100930004F1EBA2CCF01CF14BA2C4F1DA22CCF01C1
:100940004F16BA2CCF1DA72CCF014F16BA2C4F1E15
:10095000BA2CCF01CF14BA2CCF1CB12CCF014F151C
:10096000BA2C4F1DB62CCF01CF15BA2C4F1EBA2C66
:10097000CF014F15DF18E32C451EE32C471ED42C66
:10098000D01CC52CD0015015F12C501DCA2CD00103
:10099000D015F12CD01DCF2CD0015016F12C501EAB
:1009A000F12CD001D014F12C501DD92CD0015016AF
:1009B000F12CD01DDE2CD0015016F12C501EF12C44
:1009C000D001D014F12CD01CE82CD0015015F12C02
:1009D000501DED2CD001D015F12C501EF12CD00162
:1009E0005015DF181A2DC51E1A2DC71E0B2DD11C30
:1009F000FC2CD1015115282D511D012DD101D115EE
:100A0000282DD11D062DD1015116282D511E282D1E
:100A1000D101D114282D511D102DD1015116282D91
:100A2000D11D152DD1015116282D511E282DD10172
:100A3000D114282DD11C1F2DD1015115282D511D48
:100A4000242DD101D115282D511E282DD10151154C
:100A5000DF18522D451F522D471F432DD21C342D18
:100A6000D2015215DF13602D521D392DD201D2153E
:100A7000602DD21D3E2DD2015216602D521E602DCA
:100A8000D201D214602D521D482DD2015216602D74
:100A9000D21D4D2DD2015216602D521E602DD20155
:100AA000D214602DD21C572DD2015215602D521D2B
:100AB0005C2DD201D215602D521E602DD20152152F
:100AC000DF188B2DDF1B8B2DC51F8B2DC71F7C2D9A
:100AD000D31C6D2DD3015315992D531D722DD301A8
:100AE000D315992DD31D772DD3015316992D531E50
:100AF000992DD301D314992D531D812DD301531654
:100B0000992DD31D862DD3015316992D531E992D42
:100B1000D301D314992DD31C902DD3015315992DA6
:100B2000531D952DD301D315992D531E992DD30106
:100B30005315E7214008C4004108C5005F18DF14C1
:100B40005F1CDF104808C9000C304A05031D051260
:100B50000C304B05031D85120C304C05031D051090
:100B60000C304D05031D85100C304E05031D8710FC
:100B70000C304F05031D07110C305005031D0710E5
:100B80000C305105031D87120C305205031D07124E
:100B90000C305305031D871149080E020318FC2D64
:100BA00012304A05031D051612304B05031D85162C
:100BB00012304C05031D051412304D05031D85141C
:100BC00012304E05031D871412304F05031D071503
:100BD00012305005031D071412305105031D8716EE
:100BE00012305205031D071612305305031D8715D9
:100BF000FF304802031908008F08031D08009820E1
:100C000049080E02031CFC2D18304A05031D05126D
:100C100006304A05031D051618304B05031D8512C5
:100C200006304B05031D851618304C05031D0510B5
:100C300006304C05031D051418304D05031D8510A5
:100C400006304D05031D851418304E05031D871011
:100C500006304E05031D871418304F05031D07117C
:100C600006304F05031D071518305005031D0710EA
:100C700006305005031D071418305105031D871257
:100C800006305105031D871618305205031D071243
:100C900006305205031D071618305305031D871132
:0A0CA00006305305031D87150800F8
:084000000700030003000900A2
:02400E00CC33B1
:10420000010003000300030003000200020002009B
:104210000200000000000000000003000300FF0097
:10422000020000000000000000000000000000008C
:104230000000C000C000C000C000C000C000FF00FF
:10424000FF00C300F300CF00FF00C300F300CF0066
:10425000FF00C300F300CF00FF00C300F300FF0026
:104260000100FF00FF00FF00FF00FF00FF00FF0054
:10427000FF00FF00FF00FF00FF00FF00FF00FF0046
:10428000FF00FF00FF00FF00FF00FF00FF00FF0036
:10429000FF00FF00FF00FF00FF00FF00FF00FF0026
:1042A000FF00FF00FF00FF00FF00FF00FF00FF0016
:1042B000FF00FF00FF00FF00FF00FF00FF00FF0006
:1042C000FF00FF00FF00FF00FF00FF00FF00FF00F6
:1042D000FF00FF00FF00FF00FF00FF00FF00FF00E6
:1042E000FF00FF00FF00FF00FF00FF00FF00FF00D6
:1042F000FF00FF00FF00FF00FF00FF00FF00AA001B
:00000001FF
